:030000000219FDE5
:03000B000200AA46
:03002B000201656A
:03005B000202F8A6
:030073000202DEA8
:1000800002030406080C10182030406080040608A3
:100090000C10182030406080A0C000070F1F3F0DDB
:1000A0000D04050D050305030302C2AFC0D0C0E077
:1000B000206217E5256002E473E525F4F58A758B67
:1000C00000D262D0E0D0D0D2AF3285268AC262E5BB
:1000D00026F46035306803207210758B00D0E0D0B4
:1000E000D0D292D291D290D2AF32D292D291D2903B
:1000F000206E0C2066097405D5E0FDE57E42907502
:100100008B00D0E0D0D0D2AF32758A00C28DD262DF
:1001100001FF01B9306805206602C29201B930685A
:1001200005206602C29101B9306805206602C290BE
:1001300001B9C29530680A2066077403D5E0FDC294
:100140009201B9C29430680A2066077403D5E0FDB5
:10015000C29101B9C29330680A2066077403D5E0E2
:10016000FDC29001B9C2AFC2AD53E6EFC0D0C0E04E
:10017000D2D3D2AFC2CEE52A6007207449152A2116
:10018000C67800790020742EE580307E01F430E7D7
:100190000278FF53DACF207E0343DA20307E034318
:1001A000DA10C2D8C271E580307E01F430E70279FE
:1001B000FFC3E89970CB306103752A18207403756A
:1001C0002A18885FD27020740DE52B6004152B214E
:1001D000D643DA01C2D82070024134A85F20610200
:1001E000C2702074367982B70431C3E894F04003BA
:1001F00074F0F8E8C4540F28F87984B70302411B5F
:10020000C313C3138721200802C313200A06C3C8DF
:1002100098F8411B28F8500374FFF88822E52D5404
:10022000066011E533C313C31324062522F52250BB
:10023000037522FF7882B60459852224A824C3E5D9
:100240002495644002A864C3E895664002A86688C5
:1002500025E56970024185C3E8AA699A5003E8FA66
:10026000E4F9EAC333FBE56BF45B29400D256AF83A
:10027000E56A6002156A400B41850AC3E56A9A5037
:1002800002056A78FF8826C26EC3E52694F840020C
:10029000D26EC3E52594404002D26420CF0AD0E05C
:1002A000D0D043E610D2AD32C2CF053A7801E52A6C
:1002B0006005307402152AC3E55F9401400575623C
:1002C0000041D4756300756C00E5622401F562504D
:1002D000037562FFD0E0D0D043E610D2AD32C2AF9A
:1002E000C0D053E67FC260759100855694855795BE
:1002F000759104D0D0D2AF32C2AF53E6EFC2ADC0D9
:10030000D0C0E0C0F0D2D3D2AFA8FBA9FCC2D83095
:100310007102615F53DACF207E0343DA10307E032F
:1003200043DA20D271E580307E01F420E7026136A5
:1003300088278928A18653DACF207E0343DA20302C
:100340007E0343DA10C2D8C271307402A172780001
:10035000E580307E01F430E702A172885FA15A5334
:10036000DACF207E0343DA20307E0343DA10C271F5
:10037000206102813853DACF207E0343DA10307EC9
:100380000343DA20C2D8D271885A895BC3E89558F2
:10039000F8E99559F97B007E087A00C3E8948CE966
:1003A00094005005755E00812A882178A2E6A82174
:1003B0006055C3E894C8E994005008E4D2E4FB7A9D
:1003C0000A8105C3E89468E994015008E4D2E3FB8C
:1003D0007A0F8105C3E894D0E994025008E4D2E290
:1003E000FB7A1E8105C3E894A0E994055008E4D285
:1003F000E1FB7A3C8105C3E89498E994085008E44D
:10040000D2E0FB7A787E00C3E8955CFCE9955DFD5F
:1004100030E70AECF42401FCEDF43400FD755E00D5
:10042000C3EC9AED9E5003755E01885C895D855A28
:1004300058855B597802A15AC3E89527F8E99528B1
:10044000F9307C02A13E307B02A13E307A02A13716
:10045000207502815BE9FDE8FC817AE9C313F9E8C4
:1004600013F8307902A137E9C313F9E813F83078AB
:0F04700002A137E9C313FDE813FC206126C3EC9A
:10047F00941CED940240028191ED7018C3EC94C866
:10048F0050120529C3E529940A5002A172755F0025
:10049F00D270A172E529600215297888E6F97400F7
:1004AF00207F087896B90302789EE624FAFEE4349A
:1004BF0000FFC3EC9EFCED9FFD9208B90310A2084C
:1004CF005007207609D27681DD307602C276A208F7
:1004DF005016B9030DECF42401FCEDF43400FD02C9
:1004EF0004F778007900A13EB90315EC33FCED3326
:1004FF00FDC3EC940AFCED9400FD50047C007D00DC
:10050F00C3EC94FFED9400400678FF7900A13EEC18
:10051F008575F0A4C5F0A2F733F879004003020502
:10052F005A78FF790002055AE9C313F9E813F83036
:10053F007C0EE9600278FFC3E81338F8E43400F961
:10054F00C3E894FFE99400400278FF885FD27020DF
:10055F006102A172741FF4552F4BF52FC274EB700B
:10056F0002D274752A18307403752A0A306102A1F9
:10057F008620740353DAFE207403752B06D0F0D057
:10058F00E0D0D0D2AD43E6103279010205B679033F
:10059F000205B6790A0205B6791E0205B67964021C
:1005AF0005B679C80205B67817E4D5E0FDD8FAD9B3
:1005BF00F6227A147B780205DD7A107B8C0205DD3A
:1005CF007A0D7BB40205DD7A0B7BC80205DD79025B
:1005DF00B27DE4C294D5E0FDC291D5E0FDD291D5B4
:1005EF00E0FDD294D5E0FDC292E576D5E0FDD29242
:1005FF007496D5E0FDD9D9EAF8D5E0FDD8FBDBCE6E
:10060F00C29422C37C007D0075F00005F0EA33FA36
:10061F00EB33FB50F6EB13FBEA13FAC3E9FFE8FEEB
:10062F00E89AF8E99BF95004EFF9EEF8B3EC33FCD4
:10063F00ED33FDD5F0DFEDF9ECF822E889F08A20F3
:10064F00D2D4F8A9F07B0030F70B7BFFF42401F82C
:10065F00E9F43400F9E88520F0A4ADF0F8E985203D
:10066F00F0A4AFF0FEED2EF974003FFA7C04C3EA5C
:10067F0013FAE913F9E813F8DCF48BF030F70AE812
:10068F00F42401F8E9F43400F9E889F0C2D4F8A9A8
:10069F00F0227882B604030206FCC3E55F940140A2
:1006AF00030206C6852224E4F545F546F547F548CD
:1006BF00F549C26D0206FC7882E6FCD26DE522F5A3
:1006CF0023783879C7AA40AB41C3EB13FBEA13FA7F
:1006DF00EC146013C3EB13FBEA13FAEC141460076A
:1006EF00C3EB13FBEA13FAD1128845894622C3E5FF
:1006FF00459523F8E5469400F9500CC3E89480E93A
:10070F0094FF401602072DC3E8947FE9940050032D
:10071F0002072D787F790002072D788079FF884AAC
:10072F00894B22E54A2547F8E54B3548F9854B209B
:10073F00E4300701F43549FA30E709C3EA94F04091
:10074F001502076BC3EA940F500302076B78FF790A
:10075F00FF7A0F02076B780079007AF0C3E52495D2
:10076F0064500AC374019524500B020789E54B208E
:10077F00E70E020789E54B30E706884789488A4923
:10078F002278A4E6FAC3E54A33F8E54B33F9D14AA8
:10079F00E930E70BC3E89480E994FF4013E1C3C34A
:1007AF00E8947FE994005002E1C3787F7900E1C3B8
:1007BF00788079FFE820E715C3E52398F84009C34F
:1007CF00E8940140030207EA78010207EAE8F424FB
:1007DF00012523F840030207EA78FF884C2278A509
:1007EF00E6FAA848A949D14AE930E70CC3E89401D1
:1007FF00E994FF401602081EC3E894FFE9940050E5
:10080F000302081E78FF790002081E780179FFE9BC
:10081F0020E715C3E54C98F84009C3E8940140035D
:10082F000208457801020845E8F42401254CF840F8
:10083F000302084578FF88242278FFC26420693DAF
:10084F00206A12D264C3E541940A4009C3E5259496
:10085F00405002C26479A1E76023E541601F74FF35
:0F086F008541F0848539F0306A0375F005A4F8EF
:10087E00C5F0600278FFC3E895675002A8678866E6
:10088E0022C3E5409440E5419401E566500314010E
:10089E00A0046002F566220208A82275E89022786C
:1008AE0083E6FFE5E820ECF7A8BDA9BE0573C3E516
:1008BE007394084052757300E9FA79A0E76044EA30
:1008CE007007E574601B0208E3C3E895746010E5D9
:1008DE00745006600C140208EF0460F90208EFE58C
:1008EE0074F574C3946D401B7564C0C394044013B7
:1008FE00756480C39404400B756440C39404400334
:10090E0075640075BB0622E5642410500274FFF571
:10091E00647982B70402213CC3A864E5249850028E
:10092E00A824C3E895664002A86688258826E57344
:10093E00B4070375BB1022743279A687F0A4C5F0F4
:10094E00A2F733F8C3E895644002A864882288248D
:10095E00882588268867227540007541F022C2AF2F
:10096E0075C820A8CCA9CDAA3A30CF010A75C824E3
:10097E00D2AFAB3BAC3C883B893CC3E89BF8E99CCF
:10098E00206908F9306702418121DEAD3D8A3DF9CB
:10099E00EA9DFA600478FF79FFAE3EAF3F8B3E8C46
:1009AE003FC3EC9FFCC3E99CF542A83BA93CC3E8BE
:1009BE009EF8E99FF9C3E54113FBE54013FAE82AD7
:1009CE00F540E93BF54150067540FF7541FF412862
:1009DE00AA40AB41AC40AD417E047F02C3EB940410
:1009EE0040021E1FC3EB940840021E1FC3ED13FDF1
:1009FE00EC13FCDEF7C3EA9CFAEB9DFBEF6009C338
:100A0E00E913F9E813F8DFF7EA28FAEB39FB8A4025
:100A1E008B4150067BFF8B408B41C3EB94025002FF
:100A2E00D2673069047F0341537892E6FFC3E537FE
:100A3E00948240110FC3E53794A040010FC3EF9489
:100A4E000640027F057E04E541C4540FF9E541C41A
:100A5E0054F0F8E540C4540F28F8C3E89EFAE99420
:100A6E0000FB4009C3EA9402EB940050047A02E4BE
:100A7E00FB41CDAA40AB41EBC4FEEAC4540F4EFC81
:100A8E00C3EA9CFAEB9400FBC3E813C313F8EA28FD
:100A9E00FAEB3400FB8A408B41C3EB94024002C256
:100AAE00677804EBC4FE7B00EAC4540F4EFAC3EA27
:100ABE0098FA4005C3940250027A027892E6FF300B
:100ACE00600241CD855256855357D26043E680C3AE
:100ADE00E49AF8E49BF93067026167E8FAE9FBD320
:100AEE00E913FDE813FC88528953C3EF9403603871
:100AFE00EF20E00DE82CF8E93DF9ECFAEDFB020BE6
:100B0E0022E828F8E939F9C3E82402F8E93400F9B3
:100B1E007AFE7BFFC3EF9403400E8A548B55884EAA
:100B2E00894F8C508D51619B885489558A4E8B4FBD
:100B3E008C508D51306920C3E53394034019E54242
:100B4E00A2E713F8E555F4240138400B20E70875A9
:100B5E0054FFF42401F555619BE8FAD3E813FC88A1
:100B6E0052C3EF94036020EF20E007E82CF8ECFA74
:100B7E006187E8282402F87AFEC3EF940340088ABE
:100B8E0054884E8C50619B88548A4E8C50E56BC3B2
:100B9E00335002646BF56B30600261A5753402D27E
:100BAE006043E680E52D54066026A840A941C3E9BE
:100BBE0013F9E813F8C2AF53E67F759100C3E498BA
:100BCE00F594E499F595759104D26043E680D2AF21
:100BDE0022D265754400752000306B0375204002EB
:100BEE000BFED265754400752040306B03752000F6
:100BFE00D2AF7801206722E52D54066002C265C38C
:100C0E00E541940540137802940540087803940555
:100C1E0040027806306902780A206019E5446015B2
:100C2E0030690AC3E53394034003D53406D2AFD2FC
:100C3E006C81D071ADD2AF0000C2AF206726E54106
:100C4E00C3FB940F40027B0FEB240530730123305E
:100C5E006A02742820620123F93069027982E58BD9
:0E0C6E00C39940B50544E59BF45440B52002FF
:100C7C0081BA30690A08C3E8940A40010881272028
:100C8C00650261FEC26553E67F7591003067107591
:100C9C0094007595FE759104D26043E68061FEAEBA
:100CAC0040AF41C3E49EF594E49FF59581A1C3E563
:100CBC00339402500261FE30650261FED80281CE8F
:100CCC008127C26C53E67F759100855494855595A8
:100CDC00759104854E56854F57D26043E680D2AF4E
:100CEC00E52D54066008206A020533020D0A306CAB
:100CFC000D206B0A20650715811581021575227868
:100D0C00003064053065027801E53775F007A4F909
:100D1C00E5F028F5F0E9A2F013A2F113A2F213F515
:100D2C0037C394785003753778C3E5379538400846
:100D3C00D266D292D291D290306002A144855056A4
:100D4C00855157D26043E68022207D11C2AF754396
:100D5C0002C294D295D2AF759F11020F24C2AF7507
:100D6C004302C294D293D2AF759F11020F243072FA
:100D7C0043207D20C2AF754303900143757E10D292
:100D8C0090C293306204C291A198D294D2AF759F55
:100D9C0001020F24C2AF754303900143757E10D23C
:100DAC0092C295306204C291A1B8D294D2AF759F11
:100DBC0021020F24207D17C2AF75430390011ED270
:100DCC0090306202C291D2AF759F01020F24C2AF64
:100DDC0075430390011ED292306202C291D2AF755C
:100DEC009F21020F24207D11C2AF754304C295D2FE
:100DFC0093D2AF759F21020F24C2AF754304C293E7
:100E0C00D295D2AF759F01020F24307243207D2002
:100E1C00C2AF754305900132757E20D291C29430D9
:100E2C006204C292C134D295D2AF759F11020F24C5
:100E3C00C2AF754305900154757E08D291C29430AF
:100E4C006204C290C154D293D2AF759F11020F2489
:100E5C00207D17C2AF754305900114D29130620208
:100E6C00C292D2AF759F11020F24C2AF7543059089
:100E7C000128D2913062EBC290D2AF759F11020F54
:100E8C0024207D11C2AF754306C293D294D2AF75A4
:100E9C009F01020F24C2AF754306C295D294D2AF04
:100EAC00759F21020F24307242207D20C2AF754302
:100EBC0001900154757E08D292C295306204C290A2
:100ECC00C1D0D293D2AF759F21020F24C2AF75430C
:100EDC0001900132757E20D290C293306204C2928E
:100EEC00C1F0D295D2AF759F01E124207D16C2AF1F
:100EFC00754301900128D292306202C290D2AF7534
:100F0C009F21E124C2AF754301900114D29030624D
:100F1C0002C292D2AF759F01C26622900112757EF9
:100F2C0000D292D291D290C295C294C293C2622244
:100F3C00788076090876090876040876FF08760327
:100F4C000876FF08760A0876030876010876017899
:100F5C008C76010876FF0876FF0876FF0876FF0886
:100F6C0076FF0876030876FF0876FF0876FF08768A
:100F7C00250876D00876280876500876040876FF7F
:100F8C0008760208760008767A0876FF087601085B
:100F9C007601087600087603227887E6FFC272BFD6
:100FAC000302D2727888E6C394036008C27DE630EF
:100FBC00E102D27DC27E7889E630E102D27EC3EFB7
:100FCC0094026008758E01D273020FDD758E00C21B
:100FDC0073227880E6149000809378A4F67881E6EA
:100FEC00149000809378A5F67886E61490008D9383
:100FFC0078A6F6789CE67538FF75390CB402067540
:10100C0038A075390AB4030675388275390578A38A
:10101C00E61490009A93F569120F2722227896E62F
:10102C00FA7897E6FB7888E6B40305C3EB940EFBDD
:10103C00307F047A007BFFC3EB9AFCC3948250028E
:10104C007C827575000575EC8575F0A4C3E5F0948C
:10105C007D40F222D27F11291205A77A007B007CF9
:0E106C001012059DE55F2AFA74003BFBDCF3D1
:10107A007C04C3EB13FBEA13FADCF7FEC27F1129E7
:10108A0022E5EF20E6037520000520903FFFE520CA
:10109A00146006901DFF1460009304600375EF123C
:1010AA0053D9BF7581C043FF8012059875EF02437B
:1010BA00B203E5B3240420E70DF521E5E320E006B9
:1010CA008521B343E301120F277580FF75A40075CC
:1010DA00F19075D47F75900775A53F75F23F75D568
:1010EA000075A60175E241E4F8F6D8FD756B0112A8
:1010FA000F3C1215B778988676753001C2AF120583
:10110A00B11205C11205A71205C81205A71205CF0B
:10111A001205A7C2AF78FA79FA308707D9FBD8F750
:10112A00021C00120FA5120FDE11281129789886C9
:10113A0076120F2775885075891275C8247591041F
:10114A0075D84075A82275B80275E690759B8075AA
:10115A009D0075D10E75BC5875BB0675BA1175E838
:10116A0080120598D2AF1208A553DACF207E034326
:10117A00DA20307E0343DA1043DA01C2D8C2711290
:10118A0005B1D2617B037A0CE55E70077A0CDB034A
:10119A0002111D1205A720700302111DC270E55F1E
:1011AA00C3940240E1E52F541F856160F561B56083
:1011BA00D5DAD5C26153DACF207E0343DA20307EF6
:1011CA000343DA10C2D8C27178A2E67008D274E575
:1011DA002F54E0F52FC2757529001205AC30740939
:1011EA00C3E529940A4002D27512059D780230742B
:1011FA00027800C3E55F9840F0C2AF1205C112053C
:10120A00C11205C1D2AF1205B1754D007888E6B496
:10121A00030241F412059D788CE6C394015003023F
:10122A0012F4E530C3940150030212F4207435C35A
:10123A00E55F94FF50030212F4C2AF1205D6D2AF93
:10124A001205ACC3E55F940150EFC2AF1205C1129B
:10125A0005A21205C1D2AF1205ACC3E55F94FF40E7
:10126A00E902175F7F02D27F11291205ACC2AFC211
:10127A007F1129AE5FC3E55F947FD2AF4076120536
:10128A0098C2AF1205D6D2AFDFDC1160C3EE940567
:10129A007897F61205B11215F91216E27F0AD27F73
:1012AA0011291205ACC2AFC27F1129AE5FC3E55F37
:1012BA00947FD2AF50E6120598C2AF1205C112054B
:1012CA00A21205C1D2AFDFD61160EE24057896F6D8
:1012DA001205B11215F91217111205AC1129C3E53D
:1012EA005F94FF5002413602175FC3E55F954D4098
:1012FA0003855F4D1205AC78017988E7B40302785B
:10130A0005C3E55F9840024116C2AF1205D6120521
:10131A00D61205D6D2AF1205B1753000E4F531F513
:10132A00320531E531F470390532789AE6781914C4
:10133A006012783214600D787D14600878FA1460AF
:10134A0003753200C3E53298401715327531B47807
:10135A00998676C2AF1205D6D2AF789886761205EC
:10136A00AC1205A2E52A7005307402211D7801200D
:10137A0074027806C3E55F9840A77888E6C39403A9
:10138A0060031205ACE52A700302111DC2AF120FE9
:10139A0027E4F522F523F524F525F526F56AD2AFDB
:1013AA007885E6C333F568E4F545F546F547F5482B
:1013BA00F549F573F52CF52DF53775730875BB10DE
:1013CA001205981208A9E5E820ECFBA8BDA9BEE918
:1013DA007001F888741208AD75730875BB107887A8
:1013EA00E6FE7602120FA57887EEF6C2AF7564FFA5
:1013FA00120945852264852265852266D2AF752247
:10140A000175240175250175260185636C756D01C9
:10141A007888E6B40307C27D307602D27DD268D2DC
:10142A0069753300120E8D120EB212096512096C1B
:10143A0012096512096C120965021453C2AF120F20
:10144A00A5D2AF75730075BB06120BF01206A11276
:10145A000D0B120D5512096C120BDF306D031206BB
:0D146A00FD20670312084830670312088F49
:10147700120D0B120D7A12096C120BF0306D03125C
:101487000732120D0B120DF112096C120BDF306DC2
:1014970003120790120D0B120E1612096C120BF0A5
:1014A700306D031207ED120D0B120E8D12096C121F
:1014B70008A9120BDF120D0B120EB21208AD12099A
:1014C7006C306935206B3285676485676585636C29
:1014D700756D0179187A0CC3E53399400FC269D24B
:1014E7006A8A35856764856766021500C3E55F9478
:1014F70001400302145302157D306A1B206B18E567
:1015070035147004C26A8146F535C3E55F9401401E
:101517000302145302157D753600C3E56278FA9805
:101527005054307404E52A604D7888E6B4031720D8
:101537007D05207607A14D307602A14D206B07D29D
:101547006B856764819278F0306B058567647820D6
:10155700C3E5419850028153306B1BC26BC27D308B
:101567007602D27DD26A7535128567648153053656
:10157700E55F6002A180753600C2AF120F2778873A
:10158700E6FE7602120FA57887EEF6E4F522F5233C
:10159700F524F525F526F568C268D2AF120598122D
:1015A7000F27307409C3E53694054002211D6126D3
:1015B700901A0D782012163BE520B4550CA312168D
:1015C7003BE520B4AA030215D9120F3C1215F90204
:1015D70015F8901A0378807B0A12163BA308DBF9EB
:1015E700901A0F788C7B1812163BA308DBF9901A18
:1015F7002722C2AF12167A121654901A00740E12CE
:101607001640A37404121640A37414121640901ABD
:101617000378807B0A12163FA308DBF9901A0F782C
:101627008C7B1812163FA308DBF912168D12166B66
:10163700901A2722E493F622E6438F01538FFD7514
:10164700EF0275B7A575B7F1F0538FFE22438F02EE
:10165700438F0175EF0275B7A575B7F1901A0DF0B5
:10166700538FFC22901A0D7455D140901A0E74AA0C
:10167700D140227A3079D07820901A40D13BE520AA
:10168700F709A3DAF7227A3079D0901A40E7D140E8
:1016970009A3DAF922AB77A878BB01027980BB02EC
:1016A700027981BB03027982BB04027984BB0502FC
:1016B7007986BB06027992BB07027987BB08027954
:1016C700A3BB0902799CBB0A027988BB0B02798903
:1016D700E8F7227C051205B1DCFB22C2AF1205C177
:1016E7001205C81205CF1205D61205A21205C1129E
:1016F70005C81205CF1205D61205A21205C112059B
:10170700C81205CF1205D6D2AF22C2AF1205D61224
:1017170005CF1205C81205C11205A21205D612057A
:10172700CF1205C81205C11205A21205D61205CFA0
:101737001205C81205C1D2AF22AE77AF78C2AF1279
:1017470005C11205C11205C11205A2DEF21205D6A6
:101757001205A2DFF8D2AF22D1E2D1DAD1DA75775A
:1017670001757801757900F1407C05AD5F1205B10F
:10177700C3ED955F70F5C3E55F9401400AC3E55F6C
:1017870094FF403202179BD19CB1F9D1E2C2AF75E9
:10179700EF12D1DADCD50579C3E5799403500280DD
:1017A700C6D1DA0578E5771490009F93F808C3E56A
:1017B7007898500280AED1DAD1DA0577C3E577940D
:1017C7000C5002809C120F3CB1F9C2AF75EF12D1D9
:0117D700DA37
:0319FD0002108B4A
:101A00000E0414090904FF03FF0A03010155AA018A
:101A1000FFFFFFFFFF03FFFFFF25D0285004FF0259
:081A2000007AFF01010003FF41
:101A400023454D41584E616E6F3230412320202096
:101A500023424C48454C4923463333302320202031
:101A60002020202020202020202020202020202076
:101C0000C2AFC2D353D9BF7581C043B20343FF8073
:101C1000752438752503B1C975EF0275E24043F1AB
:101C20008053A47F75D400D2877DFA780379E67C4F
:101C300010752200752300901DD67B0675249875BB
:101C400025013087028142208708D8FBD9F9DCF7CB
:101C500081B4308708D8FBD9F9DCF781B4B189E4C5
:101C600093A3C39A6004DDC381B4DBDBB17B600264
:101C7000812B7B08E493FAA3B15CDBF87A30B15C8A
:101C8000752200752300B17BEAFCEBFDC3ED94FEE9
:101C9000400EB17B8A278B28ED30E0048A828B834B
:101CA000B17B7AC270D8C3ED94FE601350CEBD00F4
:101CB00025EC60097520007521FF0200008100A855
:101CC00027A9280809D804D90281D3B17FEA89AAB3
:101CD000F281C50D81A0C3ED94035049EDA2E092BD
:101CE000007AC5C3E5829400E583941C50902000DF
:101CF00010438F02438F0175B7A575B7F1F030001F
:101D00001FA827A9280809438F01538FFDD804D99C
:101D100002A12089AAE275B7A575B7F1F0A3A10DBC
:101D2000538FFC817C7AC1BD030CE493A3FAB140CC
:101D3000DCF8B138817C817EAA22AB23B15CEBFA5E
:101D4000EA6222752608C3E52313F523E52213F57D
:101D50002250066323A0632201D526EAB1C9B1C986
:101D600075260AEAF4200102D287300102C287B147
:101D7000C9C3134002C201D526EB22B17FEAFB2082
:101D80008702A17F308702A184752608AE24AF2583
:101D9000C3EF13FFEE13FEB1CDB1C9C3EA13308711
:101DA000024480FA30E703632201C3E52313F523DD
:101DB000E52213F52250066323A0632201D526D91C
:101DC000E52265236523F52222AE24AF250E0FDE22
:101DD000FEDFFCD20122424C48656C693437316326
:041DE000F3300601D5
:00000001FF
